S00C0000474C43442E73726563FE
S113000045C000004BC0000049C0000047C00000CC
S113001045C0000043C0000041C000003FC00000D4
S11300203DC000003BC0000039C0000037C00000E4
S113003035C0000033C0000031C000002FC00000F4
S11300402DC000002BC0000029C0000027C0000004
S113005025C0000023C0000021C000001FC0000014
S11300601DC000001BC0000019C0000017C0000024
S113007015C0000013C0000011C000000FC0000034
S11300800DC000000BC0000009C0000011241FBEF9
S1130090CFEFD0E1DEBFCDBF36D038C0B1CF20E046
S11300A030E008C0E3ECF9E03197F1F700C000005C
S11300B02F5F3F4F28173907ACF308958FEF84BBA8
S11300C087BB88B38B6088BB84E190E0E8CF089558
S11300D088B3806188BB81E28A95F1F7000088B318
S11300E08F7E88BB81E28A95F1F70000089588B37A
S11300F08E7F88BB88B38D7F88BB8FEF88BB8EE1F2
S113010085BBE6CF0895DADFF2DFFFCFF894FFCFA7
S9030000FC
